:1000000017C024C023C022C021C020C01FC01EC0F2
:100010001DC01CC07C919EA6AEFFA1A3A3A1A3A35B
:10002000A30850FE04000000000000001B5AFF005F
:1000300011241FBECFE9CDBF10E0A0E6B0E001C0A3
:100040001D92AC36B107E1F7CFD09AC1D9CF26EBDC
:1000500033E003C0F9013197F1F70197D8F708951C
:1000600088EE93E0F4CFCF93C09163008C2F8F5F25
:100070008F7380936300909161009295990F907EA9
:10008000609162006295660F660F607C692B9091AB
:100090006000692B90E066D16FEF8C2F90E0CF91DC
:1000A00061C1CF931092630008C08C2F90E052D1B1
:1000B0008F3F41F4CF5FC0936300C0916300C034B1
:1000C000A0F30EC0982F9F709093600085FB992736
:1000D00090F99093610086FB882780F980936200F5
:1000E000CF91089580916100811112C084E08093C6
:1000F00066008BE290E090936A008093690084E24E
:1001000090E090936800809367008DE190E011C0CB
:1001100083E08093660088E290E090936A00809389
:10012000690081E290E090936800809367008AE123
:1001300090E09093650080936400809166008093C6
:100140006B000895811104C0611102C091EA9FBD46
:1001500089BD66BF089590E0E0916400F09165006C
:10016000E80FF91FE491EFBDE0916700F09168009E
:10017000E80FF91F6491E0916900F0916A00E80FBF
:10018000F91F8491DFCF369A3699FECF85B1089555
:100190001F93CF93DF93C82F14E1D1EA0CC019BC91
:1001A00016BF84E690E053DFDFBD19BC16BE80E9C0
:1001B00091E04DDFC150C111F2CFDF91CF911F917E
:1001C00008951F93CF93DF93EC01888111E081277D
:1001D000888349DF82E0DCDF88818127888343DFF1
:1001E000DF91CF911F913CCFA39A83E687B986EC2C
:1001F00086B93699FECF369A3699FECFC5B1B99AEF
:10020000B89A81EA8FBD81E083BF4BDF6BDFC53BCE
:1002100080F080916C008F5F8F7180936C00809173
:1002200060008F5F8093600090916600891748F0AE
:1002300006C010926C0080916200811102C0109281
:10024000600011DFBB9AC39AA29A81E687B986EC57
:1002500086B9369AC0E0D0E01FEF81EAF82E80918F
:100260006000E0916900F0916A00E80FF11D0491CF
:1002700090916C00903160F0F3DE10926C0010925F
:10028000600081E690E09DDF82E690E09ADF32C078
:100290000D3F59F419BD16BE82E390E0D8DEFFBCD5
:1002A00019BC16BE82E390E011C00C3F89F404E053
:1002B00019BD16BE85E090E0CADE19BC16BF81E408
:1002C00090E0C5DE0150A1F780ED92E0C0DE12C0E3
:1002D00042DFDF5FD93748F00F3F39F48091660085
:1002E00082508093600037DFBEDE84EF91E0AFDEA6
:1002F00010926C00809161008111B1CF349BAFCF1F
:100300002F9925C0CF5FC83018F1C091600080914F
:100310006600C81798F4CC2311F0C15010C0FFBC80
:1003200019BC16BE85B7877E806185BF85B78062A0
:1003300085BF889585B78F7D85BF01C0C2E08C2FB2
:100340000ADFC09360008FDE8AEF90E080DEC0E0BD
:10035000369A85CFE199FECF1FBA8EBBE09A9927D6
:100360008DB30895262FE199FECF1CBA1FBA8EBB1C
:100370002DBB0FB6F894E29AE19A0FBE019608954C
:04038000F894FFCF1F
:00000001FF
